:1000000083018B018A01850186018C019D018F018D
:100010009001910192019301940195019801990138
:100020009A01831610308500003086008117640025
:10003000A73081008312850114309E009F019F0B21
:100040001F289E0B1F2838304B2008304B200130D2
:100050004B200C304B2006304B20C1288316FF303C
:1000600086001830850083120510851405150608D2
:1000700005118039031D2E28851083160030860057
:100080008312080096002E20851005140515160809
:1000900086000511080096002E2085100510051514
:1000A00016088600051108009B010C089C00AA2078
:1000B00003149802031867280314013099020318E7
:1000C0006728031401309A02031867281B149C0345
:1000D0001C08AA2003149902031874280314013081
:1000E0009A02031874281B149C031C08AA200314EA
:1000F0009A0203187D2803147E281B0C00349B01F0
:100100000C089C00AA2003109807031C92280310D7
:1001100001309907031C9228031001309A07031C31
:1001200092281B149C031C08AA2003109907031C87
:100130009F28031001309A07031C9F281B149C035F
:100140001C08AA2003149A07031CA8280314A92832
:100150001B0C00348207003400340A3400340034AD
:10016000643400340334E834003427341034013468
:100170008634A0340F344234403482070034B13422
:10018000BC3411308C0009308D008E0106309D008A
:1001900054200318D2288E0A8D03031DC82803306B
:1001A0008C02D5287F2003308C0209308D0010305E
:1001B0001D079B009B031B0884000E088E01800016
:1001C0009D0301300C07031DC82818088F00063056
:1001D0009D00003080384B200F301D078400000840
:1001E00030384220053003151D02031DF9282E303A
:1001F00042209D0BEC280F301D078400000830388A
:100200004220403080384B20203042204D30422068
:10021000483042207A304220003080384B2097010D
:100220008101000000009D010B309E0001309F0005
:10023000D530A0008B011030850083161F3085005B
:1002400083120B1D2629970A0B1129290000000093
:1002500000009E0B21290B309E009F0B21290130AD
:100260009F00A00B2129F4308E000B1D3A29970A1C
:100270000B113D290000000000008E0B3529000005
:10028000000000000000000000000000000000006E
:100290000301860010308500831617308500831215
:1002A0000B19970A0B110108990017089A009B0176
:1002B0009B0A851585110B110108031119020319F9
:1002C00058299B0A9B099B0A1B0A9800103085003D
:1002D0008316043085008312051D6F29C92900305B
:1002E000BD20031403111A02031C8829031D982939
:1002F0000130BD20031103141902031C8829031DBA
:1003000098290230BD2003141802031C882998295B
:100310000030BD208F001A0893000130BD209000EE
:10032000190894000230BD20910018089500A729F3
:100330000030BD2093001A088F000130BD209400CA
:10034000190890000230BD2095001808910015088A
:10035000031491020318B629031401309002031804
:10036000B629031401308F020318B62914080314A8
:1003700090020318C029031401308F020318C0290A
:1003800013088F020F089A001008990011089800AE
:10039000E7290230BD2003109807031CD929031058
:1003A00001309907031CD929031001309A07031C57
:1003B000D9290130BD2003109907031CE42903103B
:1003C00001309A07031CE4290301BD209A07C128C4
:00000001FF
